:1000000010C028C027C026C025C024C023C022C0DD
:1000100021C020C01FC00CC11DC01CC01BC01AC005
:1000200019C011241FBECFEDCDBF10E0A0E6B0E097
:10003000E8EBF5E002C005900D92A436B107D9F7C0
:1000400020E0A4E6B0E001C01D92A636B207E1F7B9
:1000500068D1B0C2D5CF80916200909163000697BD
:1000600009F443C086E090E09093630080936200BF
:1000700088E790E090936100809360002FEF86E71F
:1000800091E0215080409040E1F700C00000409195
:1000900062005091630062E381E00ED22FEF86E1AF
:1000A00091E1215080409040E1F700C000008CE3D6
:1000B00090E090936100809360002FEF86E191E1E2
:1000C000215080409040E1F700C0000084EB90E0B8
:1000D00090936100809360002FEF86E191E12150C1
:1000E00080409040E1F700C000000895BA988091E8
:1000F000620090916300039729F4B29B03C0D8D1AA
:10010000AADFC3D18091620090916300029741F40D
:10011000B29B06C0CDD148E062E381E0CDD1B5D13C
:10012000CC992DC08091620090916300029739F5BF
:1001300086E090E090936300809362002FEF81E16E
:100140009AE7215080409040E1F700C000002FEF77
:1001500081E19AE7215080409040E1F700C0000023
:100160002FEF81E19AE7215080409040E1F700C0F5
:10017000000083E090E09093630080936200089514
:10018000CF9383D101C0B2DF8AD18111FCCF8CD152
:10019000882339F0823329F0803F09F03FC001C045
:1001A000A5DF7DD18111FCCF7FD1C82F01C09EDF9B
:1001B00076D18111FCCFC13089F576D1843049F0F8
:1001C00018F48130C1F419C0853051F0873099F4AA
:1001D0000EC082E090E090936300809362000DC0B7
:1001E00083E090E0909363008093620006C060D14A
:1001F00032DF4BD113C05CD111C05AD12FEF86E74B
:1002000091E0215080409040E1F700C00000409113
:1002100062005091630062E381E04ED1CF91089576
:1002200010BE85E083BF88E582BF81E089BF089565
:100230001F920F920FB60F9211242F933F938F931B
:100240009F9388E582BF809162009091630002973E
:1002500079F48091640090916500C39794F198B30C
:1002600082E0892788BB109265001092640029C043
:100270008091620090916300039779F4809164000B
:10028000909165000697ECF098B382E0892788BBCF
:10029000109265001092640014C0809162009091E9
:1002A0006300069771F48091640090916500029755
:1002B00044F098B382E0892788BB109265001092C1
:1002C00064008091640090916500019690936500B0
:1002D00080936400B89AC09A8FEA94E00197F1F78E
:1002E00000C000008091600090916100181619060E
:1002F00074F480E090E025E12A95F1F70000019682
:10030000209160003091610082179307A4F3C09898
:100310009F918F913F912F910F900FBE0F901F9043
:1003200018952FD080E296E06BD047E060E081E046
:100330004BD080E895E273D066E080E093D070DF28
:10034000B99AD498DC9AD69ADE98789419DFFECFC1
:10035000D99840E120E030E0992314F4DB9A01C001
:10036000DB98220F331FC8992160DA9A880F991FF2
:1003700000C00000DA98415079F7D99A822F932F64
:1003800008958AB38E608ABBD99A2FEF80E792E0F6
:10039000215080409040E1F700C0000080EE90ECDA
:1003A000D7DF87ED90E8D4DF8BEA92ECD1DF81E8EC
:1003B0009AECCEDF80E090EECBDF80E098ECC8DFF7
:1003C00087EF94ECC5DF0895477050E0546963707F
:1003D000262F30E0220F331F220F331F220F331F2F
:1003E00090E0880F991F82959295907F9827807F43
:1003F00098279927822B932B842B952BA9DF08957F
:100400008036910538F080342FE0920728F08FE392
:100410009FE002C080E690E0906A9ADF08958739F5
:1004200022E09207F0F0883125E1920770F49C01F8
:1004300040E050E060E678EA80E090E0A0D0C901BA
:1004400001978068966C84DF08959C0140E050E03D
:100450006CEF72E485E090E070D0C9010197966C72
:1004600077DF0895877090E0986970E062957295E3
:10047000707F7627607F76277727862B972B68DF1C
:100480000895D998C89BFECF089588EC92E860DF64
:1004900081E89AEC5DDF83E89AEC5ADF0895D998F9
:1004A00089B380958170089580E090EB51DF0895C5
:1004B00088E092E84DDF08951F93CF93DF93182FC4
:1004C000D62FC42F88E392E843DFDBDF8AEA98EB7C
:1004D0003FDFD7DF8AEA98EB3BDFD3DF8AEA98EB8E
:1004E00037DFCFDF8DE298EB33DFCBDF84ED98EBA6
:1004F0002FDFC7DF812F90E0986B2ADFC2DF8D2FBF
:1005000090E0986B25DFBDDF8C2F90E0986B20DFAB
:10051000B8DF80E098EB1CDFB4DF88E092E818DFFA
:100520002FEF80E792E0215080409040E1F700C03B
:100530000000DF91CF911F910895A1E21A2EAA1B0E
:10054000BB1BFD010DC0AA1FBB1FEE1FFF1FA21783
:10055000B307E407F50720F0A21BB30BE40BF50B80
:10056000661F771F881F991F1A9469F76095709509
:10057000809590959B01AC01BD01CF010895052E9A
:1005800097FB16F4009406D057FD0CD0D6DF07FC7D
:1005900009D07EF490958095709561957F4F8F4F2F
:1005A0009F4F089550954095309521953F4F4F4F5F
:0805B0005F4F0895F894FFCF9E
:0405B800B400020089
:00000001FF
